:1000000000308A0004280000FF238316900000308F
:100010008A00692A2F308400000803191E28013045
:10002000A100A001A00B1228A10B11284A30A000AA
:10003000A00B182800000000800B0F28003410309F
:10004000B200A001A301AF0CAE0C031C2D28300898
:10005000A0070318A30A3108A307A30CA00CA20C45
:10006000A10CB20B23280034A101A201A001A3011D
:100070003308031D3E283208031958281030B400F5
:100080000310B00DB10DA00DA30D33082302031D05
:100090004B2832082002031C54283208A002031CFB
:1000A000A3033308A3020314A10DA20DB40B40282F
:1000B000000000340030A1001F08C33921049F0054
:1000C0000330A000A00B62289F149F1865281E080B
:1000D000AB01AA002B08AF002A08AE00B101FA302C
:1000E000B0001F202208AF002108AE002208B10096
:1000F0002108B0000330B300FF30B20034202208E2
:10010000AB002108AA0083160515003083120519DB
:100110000130013C031DAB28831687108312871022
:10012000AD01AC012D082B02031CA728031D9C2840
:100130002C082A02031CA7280430AE00FA30AF00B6
:100140000A20AE0B9E28AC0A0319AD0A922883162A
:100150008710831287148316051500308312051942
:100160000130003A031DD3288316871083128710AD
:10017000AD01AC012D082B02031CCF28031DC428A0
:100180002C082A02031CCF28F030AE00FA30AF0052
:100190000A20AE0BC628AC0A0319AD0ABA2883168A
:1001A00087108312871400348316071183120711F6
:1001B0005A208316071183120715D928BD2A8316E2
:1001C0000711831207155A2083160711831207118E
:1001D000E428BD2A0430A1001F08C33921049F0070
:1001E0000330A000A00BF2289F149F18F5281E08CA
:1001F000AB01AA002B08AF002A08AE00B101FA300B
:10020000B0001F202208AF002108AE002208B10074
:100210002108B0000330B300FF30B20034202208C0
:10022000AB002108AA0083160515003083120519BA
:100230000130013C031D3B29831607108312071070
:10024000AD01AC012D082B02031C3729031D2C29FD
:100250002C082A02031C37290430AE00FA30AF0004
:100260000A20AE0B2E29AC0A0319AD0A22298316E7
:100270000710831207148316051500308312051921
:100280000130003A031D63298316071083120710FB
:10029000AD01AC012D082B02031C5F29031D54295D
:1002A0002C082A02031C5F29F030AE00FA30AF00A0
:1002B0000A20AE0B5629AC0A0319AD0A4A29831647
:1002C00007108312071400348316071183120711D5
:1002D0005A208316071183120715EA206429BD2AC4
:1002E00083160711831207155A20831607118312EC
:1002F0000711EA207029BD2A1430A800FA30AF0097
:100300000A20A80B7E2983168715003083128719CF
:100310000130A8008316871600308312871A013037
:100320002805A100211896292710972927140030A5
:1003300027180130A8008316071600308312071E05
:1003400001302805A1002118A729A710A829A71462
:10035000A718B42983160711831207115A20831690
:10036000071183120715EA208329BD2A1430A8003B
:10037000FA30AF000A20A80BB82983168715003081
:10038000831287190130A800831687160030831264
:10039000871A01302805A1002118D0292710D1295A
:1003A0002714003027180130A800831607160030E4
:1003B0008312071E01302805A1002118E129A7108A
:1003C000E229A714A718F22983160711831207152B
:1003D0005A208316071183120711EA20831607118A
:1003E00083120715BD29BD2A1430AA00FA30AF00C8
:1003F0000A20AA0BF6298316871500308312871965
:100400000130AA008316871600308312871A013044
:100410002A05A8008316071600308312071E013034
:100420002805A900A908031D262AA7012708023CC0
:10043000031C262A83160711831207115A208316DC
:10044000071183120715EA20A70A162AFB29BD2ADD
:1004500027101430A800FA30AF000A20A80B2B2A6E
:10046000831687150030831287190130A800831680
:10047000871600308312871A01302805A100211841
:10048000432AA710442AA7140030A7180130A80057
:100490008316071600308312071E01302805A100BD
:1004A0002118542A2711552A27152719672A0130A0
:1004B000A7062718602A8316071183120715EA205A
:1004C000271C672A83160711831207115A20302A26
:1004D000BD2AFF238316900084011F3083058312F9
:1004E0001F13003083169100073083129900FA30F1
:1004F000AF000A201F1300300138831691008312C9
:100500001F13003002388316910083121F1300302E
:10051000831691001F169F161F1383129F131F141B
:10052000FA30AF000A20831685158312A601851DB7
:10053000A60A0310260DA7008316051600308312A5
:10054000051E01302704A6000310260DA700831600
:10055000851600308312851E01302704A600260868
:10056000F83E0318BD2A083EBE2AD428DF28642995
:1005700070297C29B629F429282A63000A108A14D4
:100580000A118207B52AB62AB72AB82AB92ABA2A7E
:04059000BB2ABC2A9C
:02400E008431FB
:00000001FF
